:040000000FEF00F00E
:0600080004EF10F01200ED
:100018000CEF10F0120038EF0BF0080ECE6F010E47
:10002800CF6F03C1D0F006C1CDF0040E016E010EF2
:10003800026E08EC0DF001C0C8F002C0C9F0000162
:10004800D16BFF0E016EFF0E026EFF0E036EFF0EE8
:10005800046E020E056E010E066ECD51060F076E78
:10006800D5EC08F0011C576E021C586E031C596E23
:10007800041C5A6E080E0001CD25016E026A010E9D
:100088000222EDEC05F0575001180AE15850021809
:1000980007E15950031804E15A500418D8B40CD099
:1000A800060E206EC8C021F0C9C022F0D05115EC50
:1000B80005F00001906B120001010205D8B40BD0C5
:1000C800010E206EC8C021F0C9C022F00001D05135
:1000D80015EC05F0120000019051D8B412D09151DE
:1000E800D019D8A40ED07C51C8190BE17D51C9197B
:1000F800D8A407D0950E1D6E92C01EF098EC0BF098
:100108001200D005D8A407D0CD51D8B402D0020E21
:10011800ABD1D16BAAD1020ED019D8A494D08F6BD1
:10012800100ECD19D8A4F3D7CEC001F0CFC002F07D
:1001380071EC0CF00009D8B416D0040ECE25016E6F
:10014800000ECF21026E71EC0CF00009D8B40BD070
:10015800080ECE25016E000ECF21026E71EC0CF058
:100168000009D8A402D0040E7FD1CEC001F0CFC0C0
:1001780002F008EC0DF001C0C4F002C0C5F0040E96
:100188000001CE25016E000ECF21026E08EC0DF0A5
:1001980001C07AF002C07BF0080E0001CE25016E86
:1001A800000ECF21026E08EC0DF001C0C6F002C0AF
:1001B800C7F00C0E0001CE25016E000ECF21026E95
:1001C800EDEC05F001C06CF002C06DF003C06EF0FC
:1001D80004C06FF0200EC519C411D8A4C4D7C10E2D
:1001E8007A5D7F0E7B59D8B0BED77A51C45D7B51FA
:1001F800C559D8B0B8D7C651C711D8B4B4D7C451A7
:100208007A5D576EC5517B59586EC651575CC751B8
:100218005858D8A0A8D7CCEC0AF00001D16FD1511A
:10022800D8A423D1C6C078F0C7C079F0776B000E88
:10023800766F200E756F000E746F686969696A6958
:100248006B69010EF6D0030ED019D8A486D0040E1F
:10025800CD655DD7440ECD6501D059D78F05D8B48B
:1002680002D0030E01D1CEC001F0CFC002F071EC74
:100278000CF00009D8B477D7CEC001F0CFC002F097
:1002880008EC0DF001C0CAF002C0CBF00001CD515E
:10029800FC0FCC6F7451CA5D7551CB59D8A063D788
:1002A800200ECB5DD8A05FD77A51CA5D7B51CB5960
:1002B800D8B059D7CA517A5D576ECB517B59586E11
:1002C800CC51575C000E5858D8A04DD77651785D60
:1002D800576E77517959586ECC51575C000E585863
:1002E800D8B002D0080EC0D0CAC00CF0CBC00DF0F8
:1002F800040ECE250E6E000ECF210F6ECCC010F06E
:1003080083EC07F00001D16FD151D8A4AED068C0FA
:1003180001F069C002F06AC003F06BC004F0040E7B
:10032800CE25056E000ECF21066ECCC007F0D5ECA9
:1003380008F001C068F002C069F003C06AF004C0A8
:100348006BF00001CC517627000E7723CC51CA25DB
:10035800746F000ECB21756F88D0040ED019D8A405
:1003680041D0040ECD19D8A4D2D68F05D8A479D7F8
:10037800CEC001F0CFC002F0EDEC05F06C510118D1
:1003880026E16D51021823E16E51031820E16F51E7
:100398000418D8A41CD07851761919E17951771925
:1003A800D8A415D0681D576E691D586E6A1D596E00
:1003B8006B1D5A6E6C5157180AE16D51581807E1B8
:1003C8006E51591804E16F515A18D8B402D0060E6C
:1003D8004BD02BEC0EF00001D16FD151D8A445D0F1
:1003E800020E27D0050ED019D8A425D0CD51D8A4F7
:1003F8008ED6020E8F19D8A434D7200E0D6E000E9B
:100408000C6E7AC00EF07BC00FF078C010F079C087
:1004180011F06CC012F06DC013F06EC014F06FC014
:1004280015F000EC03F00001D16FD151D8A41DD014
:10043800030E8F6F1AD0060ED019D8A408D0CD514C
:10044800D8A465D6030E8F19D8A40BD70ED07F0E6B
:10045800D019D8A408D0CD51D8A459D6D0EC0DF0D5
:1004680000018F6B02D0010ED16FD1C020F0C8C03F
:1004780021F0C9C022F0D05115EC05F0060E00019C
:10048800D019D8A41200D151D8A4120028EC0EF02B
:100498001200010E196E1B6A000E1A6E85D0DA0E54
:1004A800C16F1F0EC26FC151C211D8A4000EC36F15
:1004B8001B6A120E1A6E196A85D06251D8A482D0AE
:1004C8006251020DEF0EF324F66E1E0EF420F76E45
:1004D8000900F5CF11F00900F5CF12F011C013F0A3
:1004E80012C014F0156A13C0C1F014C0C2F015C0D0
:1004F800C3F06251020DEF0EF324F66E1E0EF420C7
:10050800F76E0900F5CF11F00900F5CF12F011C010
:1005180013F012C014F0156A13C016F014C017F0C7
:1005280015C018F0020E1624F66E000E1720F76E8E
:10053800000E1820F86E0900F5CF1AF00A00F5CF62
:100548001BF0B9D7070E626501D03CD06251020D8D
:10055800DF0EF324F66E1E0EF420F76E0900F5CFB9
:1005680011F00900F5CF12F011C013F012C014F009
:10057800156A13C0C1F014C0C2F015C0C3F0C1C0E1
:10058800F6FFC2C0F7FFC3C0F8FF0800F5501A6EA7
:100598001B6A91D7C10E016E1A0E026E43EC0EF063
:1005A8000009D8A488D70ED000016351010AD8B435
:1005B80076D7030AD8B481D7010AD8B4C3D7050AB5
:1005C800D8A4E8D71950D8B407D0080E016E040E85
:1005D800026E89EC0DF012001AC001F01BC002F087
:1005E80066C003F067C004F0000E58EC0BF03BEC5B
:1005F80008F0010E896F1200200E0D180C10D8A4F7
:1006080010D0C10E0E5C7F0E0F58D8B00AD00E5015
:100618000C5C0F500D58D8B004D010501110D8A44D
:1006280002D0040E1200200E046E000E036EDAECE7
:100638000DF0FF0AD8A40BD0200E046E010E036E35
:10064800DAEC0DF0FF0AD8A402D0080E1200160E3C
:10065800016E026A000E046E0368066A400E056E9B
:100668009FEC0CF0566AD70E5624F66EF76A1E0EEB
:10067800F7225650160FD96EDA6A0800F5CFDFFF59
:10068800562A070E5664EFD71E0E016E0CC002F0F4
:100698000DC003F0046A056AEFEC0BF0220E016E40
:1006A8000EC002F00FC003F0046A056AEFEC0BF00D
:1006B800260E016E10C002F011C003F0046A056A2C
:1006C800EFEC0BF02A0E016E12C002F013C003F01B
:1006D80014C004F015C005F0EFEC0BF02E0E016EFF
:1006E800121C026E131C036E141C046E151C056E7E
:1006F800EFEC0BF0320E016EC30E026E3C0E036E71
:10070800AA0E046E510E056EEFEC0BF0360E016E5C
:100718003C0E026EC30E036E550E046EAE0E056ED1
:10072800EFEC0BF07F0E066EC00E056E160E076E10
:10073800086A8AEC08F00009D8A402D0050E120055
:10074800000E120065B464A40DD06494050E000177
:100758008A19D8A405D0609284C08AF001D0659423
:1007680065B4FDD7050E00018A19D8B4120065A03A
:1007780009D0020E8A19D8A456EC06F0030E00011F
:100788008A6F659065A807D0648460828AC084F007
:10079800050E8A6F6598030E8A6158D01200000012
:1007A800000061CF8EF0659600018E31E832E832A4
:1007B8000F0B0009D8B403D031EC0EF012008EB53F
:1007C80028D08EA302D0BB8502D00001BB958EA392
:1007D80003D01C6A1C2A01D01C6A1C50040D000E90
:1007E800F324D96E040EF420DA6EDF30E8320F0BF2
:1007F8000D0AD8A403D02DEC04F028D0020E000175
:100808008919D8A403D0BB715EEC09F012EC0AF088
:100818001DD08905D8A404D0BC713BEC08F016D0D3
:1008280012EC0AF000018B51D8B412008CC063FF9F
:10083800030E8A19D8A406D08C51D8B403D0040E5C
:100848008A6F03D08C51D8B465808B6B65A6120073
:10085800A6D70401086B00018EA30CD0240E016EEC
:10086800040E026E600E036E046A080E056ECBEC71
:100878000CF00BD01C0E016E040E026E600E036E9F
:10088800046A080E056ECBEC0CF0609812EC0AF0C6
:100898000001BB81BC816039E832030B0009D8B480
:1008A80026D048D04DEC02F01200E0EC07F0120020
:1008B800BAEC0DF012001DEC09F0120082EC05F004
:1008C8001200FAEC0DF012001BEC0DF0120059ECBE
:1008D8000CF01200F5EC0CF01200F3EC0DF0120025
:1008E800080E016E040E026E89EC0DF012006151C3
:1008F800000AD8B4E3D7010AD8B4D7D7020AD8B4C3
:10090800D4D7060AD8B4D4D7030AD8B4CBD7010AA7
:10091800D8B4D7D70F0AD8B4D7D7010AD8B4CBD709
:10092800030AD8B4D4D7010AD8B4D4D7070AD8B49C
:10093800D4D7D6D73AEC0EF00009D8A41200D0D7F5
:100948005FD0B40E016E3DEC0EF0026A070E016E28
:1009580066C003F067C004F0010E58EC0BF03BECE6
:1009680008F0010E1DEC0EF0010E1200AD0E016E26
:100978003DEC0EF0675104E1080E665DD8A002D088
:10098800000E120066C001F067C002F014EC0EF011
:10099800010E836F020E1DEC0EF0E6D7645165114F
:1009A800D8A4EED749EC0EF001EC0EF0DDD7A50E79
:1009B800016E3DEC0EF06751E3E1090E665DD8B0BB
:1009C800DFD766C001F067C002F014EC0EF0020E2B
:1009D8001DEC0EF0010E1200A50E016E3DEC0EF09E
:1009E800026A080E016E66C003F067C004F0010ECB
:1009F80058EC0BF03BEC08F0010E1DEC0EF0B4D7F0
:100A08006151000AD8B4D3D7010AD8B4E5D7210A6E
:100A1800D8B4ACD7010AD8B494D7030AD8B4BED78F
:100A2800AFD7286E020E296E540E0001956F4B0E3B
:100A3800966F010E976F2050D8B402D0810E01D066
:100A4800800E276E27C098F0990E016E21C002F023
:100A580022C003F096EC0DF02804D8A40CD0205046
:100A6800D8A409D0040E296E9F0E016E036A400EA9
:100A7800026E96EC0DF09B0E016E29C002F0036A1F
:100A880096EC0DF028C09DF020C09EF0FF0E016E80
:100A9800FF0E026EFF0E036EFF0E046E970E056EBC
:100AA800066A2950060F076ED5EC08F001C023F03E
:100AB80002C024F003C025F004C026F029509D0F81
:100AC800016E231C026E241C036E251C046E261C5A
:100AD800056E25EC0CF029500C0F0001926F28C010
:100AE80091F021C07CF022C07DF0010E906F950E30
:100AF8001D6E92C01EF098EC0BF01200010E096EEC
:100B08000A6A040E00018A19D8B43BD0060E8A1965
:100B1800D8B437D041D08DA102D00A8001D00A9034
:100B280000018DA302D00B8001D00B90096A34D04C
:100B3800060E8A19D8A407D064510F0B086E020E4E
:100B4800086401D029D0060E8A19D8B405D064519A
:100B58000F0B0009D8A420D064AF03D0086A082A74
:100B680001D0086A000164510F0B020DF350BB0F4E
:100B78000824D96EDA6ADFA202D00A8001D00A906E
:100B8800D5D760511F0B000AD8B4C5D7010AD8B40D
:100B9800CDD7030AD8B4CCD70950D8B407D0080E9B
:100BA800016E040E026E89EC0DF012002C0E016E1F
:100BB800040E026E046A080E036E000EB5EC0CF00B
:100BC8000AC02CF4020E2DEC0DF0010E0001896F05
:100BD800120020EE03F00150D9260250DA22DF502D
:100BE800056E05C006F0076A086A096A06C009F0BA
:100BF800086A076A066A20EE02F00150D9260250F8
:100C0800DA22DF500A6E0AC00BF00C6A0D6A0E6A0F
:100C18000CC00EF00BC00DF00C6A0B6A20EE01F050
:100C28000150D9260250DA22DF500F6E0FC010F0A3
:100C3800116A126A136A12C013F011C012F010C0C0
:100C480011F0106A01C0D9FF02C0DAFFDF50146E3C
:100C580014C015F0166A176A186A10501510196E24
:100C6800115016101A6E125017101B6E13501810D0
:100C78001C6E0B5019101D6E0C501A101E6E0D5064
:100C88001B101F6E0E501C10206E06501D10016E9A
:100C980007501E10026E08501F10036E09502010D6
:100CA800046E12001D0E646E666A656A676A6A6A77
:100CB800080E6B6E080E6C6E636A8D918D93150E1F
:100CC800626E000E016E040E026E046A1C0E036E44
:100CD800000EB5EC0CF0040E0401036F1C0E026F3D
:100CE800040E076F240E066F040E0B6F2C0E0A6F8E
:100CF800BB0E016E026A046A060E036E000EB5ECA6
:100D08000CF0086A0850020DF350BB0FD96EDA6A6E
:100D1800DF840850020DF350BC0FD96EDA6ADF8405
:100D2800082A020E0864EED700018B6B856B886B6E
:100D380001D0659665B6FDD76098160E6A6E8A5121
:100D4800D8A407D06086010E8A6F60BAFED7020E5B
:100D58008A6F896B608C0000000000000000609CB6
:100D680012EC0AF00001BB9512EC0AF012009DEC9F
:100D780009F00001D96FC5EC0DF06CEC0DF0000125
:100D8800D76F45EC0AF00001D86FD751D8A407D027
:100D9800D851D8B404D0D951D8B4E3EC0DF00F0130
:100DA8005B6B5C6B5D6B5E6B5F6B08EC0EF019EC5C
:100DB8000EF0F29EF29CA394D751D8A425D0D85116
:100DC800D8B422D0D951D8B41FD0D66B000ED56F65
:100DD8000ED0B7EC0BF0100E0001D36F940EE82E76
:100DE800FED7D32FFCD700000001D54BD62B300EF1
:100DF800D55D750ED659D8B003D07F51D8B4E9D790
:100E08007F51D8B4E3EC0DF0B7EC0BF00001805142
:100E1800D8B4FAD7DC51D8B4F7D7020E0001D46F92
:100E2800380ED36FAD0EE82EFED7D32FFCD7D42FB4
:100E3800FAD7FF00E9D75ED05BC0D9FF5CC0DAFF04
:100E4800DF505E6E5B4A5C2A9451D8A40ED0540ED3
:100E58005E18D8A44FD0000E9425D96EDA6A010E18
:100E6800DA225EC0DFFF942B45D09405D8A40AD0BF
:100E78004B0E5E18D8B4EFD7540E5E18D8B43AD0DB
:100E8800946B38D0000E9425D96EDA6A010EDA22F6
:100E98005EC0DFFF942B080E9419D8A41FD001015F
:100EA8000751D8A403D0440E066513D0020E206E55
:100EB800040E016E010E026E08EC0DF001C021F067
:100EC80002C022F00101035115EC05F00001906BFE
:100ED800D7D706510C0F0001936F0CD09351D8B49B
:100EE80009D093519419D8A405D011EC00F0000151
:100EF800946B936B5D065D28D8B412009DD7146A75
:100F080055D0C00E0C14156EFF0E0D14166E15502C
:100F18000C5C116E200E165CD8A006D0C00E155CB5
:100F28007F0E1658D8A002D0070E120015500001E7
:100F3800DA1904E11650DB19D8B418D040EC0CF0DB
:100F4800126E1250D8B402D012501200500E016E18
:100F5800010E026E000E046E0368066A400E056EEE
:100F68009FEC0CF015C0DAF016C0DBF014500E241C
:100F7800D96E000E0F20DA6E500E1124E16EE26A6F
:100F8800010EE222DFCFE7FF010E00017E6F3F0E68
:100F98001118D8A408D040EC0CF0136E1350D8B434
:100FA80002D013501200142A0C4A0D2A1050145C57
:100FB800D8A0A7D7000E1200010E086E040E00017B
:100FC8008A19D8B43CD0060E8A19D8B438D03FD084
:100FD80062056311D8A43BD06105D8B403D0076A71
:100FE800072A01D0076A074600018D510718FD0B33
:100FF80007188D6F086A2BD062516311D8A427D0C7
:10100800060E8A19D8A407D064510F0B076E020E7A
:10101800076401D01CD0060E8A19D8B405D06451D3
:101028000F0B0009D8A413D064510F0B0009D8A4E2
:1010380003D04EEC0DF0DED7DAEC09F0DBD76051C7
:101048001F0B000AD8B4C4D7020AD8B4D5D70850A1
:10105800D8B407D0080E016E040E026E89EC0DF0AC
:10106800120001EC0EF0030E0001896F120070C02F
:1010780010F0715104E1090E705DD8A002D0080E7D
:10108800106E70517111D8B438D08651D8A41FD0C1
:10109800C1C00DF0C2C00EF00F6A0DC001F00EC045
:1010A80002F00FC003F02C0E046E040E056E10C083
:1010B80006F0F3EC0AF010500D6E0E6A0DC0E8FF52
:1010C800C1270EC0E8FFC223000EC3230DD087C07E
:1010D80001F0026A2C0E036E040E046E10C005F0B7
:1010E800CBEC0CF01050872710502DEC0DF0105061
:1010F8000001705F000E715B12008551D8B41200B8
:10110800000E2DEC0DF00001856B120005C009F0F2
:101118003F0E0916D8A408D0200E065CD8A004D02B
:10112800800E065CD8A002D0000E120005C001F0A7
:1011380006C002F00EEC0EF00B6A0B500724D96EB5
:10114800000E0820DA6EDF50F56E0D000B2A3F0EF8
:101158000B64F3D705C001F006C002F00EEC0EF0E8
:10116800A68EA69CA698A6843EEC0DF0A6940B6AC3
:101178000B500724D96E000E0820DA6E0B50052498
:10118800036E000E0620046EDAEC0DF00A6EDE50D7
:101198000A18D8A4C9D70B2A3F0E0B64E9D7010E49
:1011A80012003AD005C0D9FF06C0DAFFDF50086E3A
:1011B8000850011A054A062A106A01B008D0000E24
:1011C8000C6E000E0D6E000E0E6E000E07D0200E77
:1011D8000C6E830E0D6EB80E0E6EED0E0F6E01C006
:1011E80008F002C009F003C00AF004C00BF0D89060
:1011F8000B320A32093208320C500818016E0D50B1
:101208000918026E0E500A18036E0F500B18046E60
:10121800102A070E1064D1D707060728D8A4C2D70A
:1012280001C001F002C002F003C003F004C004F0E2
:101238001200040E00018A19D8B404D0060E8A19C7
:10124800D8A431D063512FE1020E625DD8B02BD003
:10125800608C0000000000000000609C076A0750D6
:10126800020DF350BB0FD96EDA6ADF840750020D06
:10127800F350BC0FD96EDA6ADF84072A020E0764BE
:10128800EED701EC0EF0030E0001896F62C088F002
:101298008851D8B405D040EC0EF0060E8A6F1200C3
:1012A800040E8A6F1200080E016E040E026E89EC9D
:1012B8000DF0120072C007F0735104E1090E725D5F
:1012C800D8A002D0080E076E8EB30CD01C0E016E8B
:1012D800040E026E87C003F0046A07C005F0CBEC69
:1012E8000CF00BD0240E016E040E026E87C003F0C2
:1012F800046A07C005F0CBEC0CF0075087270750AD
:10130800725F000E735B72517311D8A412002EEC39
:101318000EF00009D8B403D001EC0EF006D0080E88
:10132800016E040E026E89EC0DF0030E0001896F48
:101338001200D0B202D0010E01D0000E076E056A6D
:101348000750D8B4D0B002D0010E056E0550D8B4FD
:1013580002D0010E01D0000E016ED0B802D0010EED
:1013680001D0000E026ED0B602D0010E01D0000EE0
:10137800036E066A0750D8A40BD00150D8A408D031
:101388000250D8A405D00350D8A402D0010E066E8E
:101398000650D8B402D0010E01D0000E046ED088D9
:1013A800D086D084D082D0800450120064AF03D09D
:1013B800046A042A01D0046A000164510F0B020D6B
:1013C800F3500424056E0528066E6105D8A40BD0D9
:1013D80064510F0B016E000E64BF010E026E0650C1
:1013E8000AEC0CF0120064AF03D0046A042A01D09E
:1013F800046A000164510F0B020DF350BB0F042463
:10140800D96EDA6ADF820650040D000EF324016EED
:10141800040EF420026E89EC0DF012000001BBA549
:1014280003D0016A012A01D0016A0150040D010E9E
:10143800F324D96E040EF420DA6E080EDF6E000174
:10144800BBA503D0016A012A01D0016A0150040D2D
:10145800000EF324D96E040EF420DA6EDF6A000160
:10146800BBA503D0016A012A01D0016A0150040D0D
:10147800000EF324D96E040EF420DA6E000EDB8E13
:101488001200200E046E000E036EDAEC0DF0FF0A57
:10149800D8A40BD0200E046E010E036EDAEC0DF00A
:1014A800FF0AD8A402D0000E1200066ADC0E062439
:1014B800036E046A7F0E0422DAEC0DF0056ECF0E7F
:1014C8000624F66EF76A1E0EF7220800F550051876
:1014D800D8A4E9D7062A070E0664E8D7010E120039
:1014E800800EB46F250EB56F000EB66F000EB76F85
:1014F800B86BB96B080EBA6F0401106B040E136F4A
:10150800340E126F146B040E176F3E0E166F186BA5
:10151800040E1B6F7E0E1A6F6B886B826C886C963C
:101528006C846C820001BE93BF93C09321EC0EF0D3
:10153800AFEC0DF00001836B120005C007F03F0E01
:101548000716D8A408D0200E065CD8A004D0800EB8
:10155800065CD8A002D0000E120005C001F006C03B
:1015680002F00EEC0EF0A68EA69CA688A6843EEC91
:101578000DF0A694A69805C003F006C004F0DAECB6
:101588000DF0FF0AD8A402D0010E1200000E1200BE
:10159800DA69DB697E6B7F0E066EC00E056EA1EC04
:1015A8000AF00009D8A402D0050E1200200E096E18
:1015B800000E086E08C005F009C006F0A1EC0AF09C
:1015C8000009D8B4F1D7400E0826000E0922C00E33
:1015D800085C7F0E0958D8A0EDD7000E12000C6ADF
:1015E8001CD00C50076E086A07500124096E085079
:1015F80002200A6E000E03200B6E09C0F6FF0AC017
:10160800F7FF0BC0F8FF0C500424D96E000E05201C
:10161800DA6E0800F5CFDFFF0C2A06500C5CD8B054
:101628001200DFD78351D8B40BD0836BB151D8A443
:1016380007D0B251D8A404D0080EB319D8B402D038
:10164800000E1200ADC0B4F0AEC0B5F0AFC0B6F039
:10165800B0C0B7F0B1C0B8F0B2C0B9F0B3C0BAF01A
:1016680047EC0EF0010E12008A0EF66E1C0EF76E95
:10167800000EF86E0900F5CFDAF00900F5CFDBF0BF
:101688000900F5CFDCF001EE00F0900EEE6AE806F6
:10169800FDE100EE68F05C0EEE6AE806FDE1000E82
:1016A800F86E0001BBEF06F0066E06C086F0035028
:1016B800015C04500258D8B010D001C070F002C0CC
:1016C80071F001C005F0070E0516D8A402D0010E6E
:1016D80001D0000E0001856F120003C070F004C035
:1016E80071F00001856B12000350D96EDA6ADFB021
:1016F80003D0066A080E02D0066A480E056E01C0BD
:10170800D9FF02C0DAFF05C0DFFF20EE01F001506B
:10171800D9260250DA2204C0DFFF01C0D9FF02C077
:10172800DAFF000EDB8E120002D0A6EC03F00001F7
:10173800DC51D8B4FAD71F6A0DD01D501F24D96EBA
:10174800DA6A7E0E1F24E16EE26A040EE222DFCF1F
:10175800E7FF1F2A1E501F5CD8A0EFD7DC6B1E5076
:10176800A3EC0DF01200A6EC03F025EC0EF05F6E72
:10177800060E5F6001D012008151D8B4120082C0F9
:10178800D2F0816B010E7F6F3E0E5B6E040E5C6EB5
:10179800D2C05DF01FEC07F0AFEC0DF0120010D0D6
:1017A800BE7148EC0EF012008EB506D0BF7115C49C
:1017B80082F034EC0EF01200C07137EC0EF012001B
:1017C8008E31E832E8320F0B010AD8B4E9D7030AA0
:1017D800D8A41200E9D70150D96EDA6A02C0DFFF37
:1017E8000150D96EDA6A010ED92603C0DFFF015015
:1017F800D96EDA6A020ED92604C0DFFF0150D96E0D
:10180800DA6A030ED92605C0DFFF1200036E015005
:10181800020DF350BB0F0224D96EDA6ADF92015031
:10182800020DF350BB0F0224D96EDA6ADF90035021
:10183800040D000EF324D96E040EF420DA6EDF6A6C
:1018480012000150D96EDA6A02C0DFFF0150D96E6A
:10185800DA6A010ED92603C0DFFF0150D96EDA6AB1
:10186800020ED92604C0DFFF0150D96EDA6A030ED2
:10187800D92605C0DFFF12007E51D8A402D0000E81
:101888001200DAC005F0DBC006F0500E076E010E3C
:10189800086E8AEC08F00009D8A402D0050E1200E0
:1018A8000001DA69DB697E6BEAD7060E00018A1946
:1018B800D8A40CD0020E646109D004012C6B010E6F
:1018C8002DEC0DF0010E0001896F1200080E016E5B
:1018D800040E026E89EC0DF01200036A20EE02F08D
:1018E8000150D9260250DA22DF50D8A40BD020EEBE
:1018F80003F00150D9260250DA22DF50D8A402D0D2
:10190800010E036E03501200026E0250D8A407D0D5
:101918000150D8A404D00001BE91010E120002505B
:10192800D8A407D00104D8A404D00001BF91C09165
:10193800F4D7000E120001C007F002C008F008D06A
:1019480007C0D9FF08C0DAFF03C0DFFF074A082A2B
:101958000506D8A006060528F3E10628D8B4120023
:10196800EFD7056E076A000E066E0AD006500124EE
:10197800D96E07500220DA6E05C0DFFF064A072A33
:101988000350065C04500758D8B01200EFD7066A17
:101998000FD006500124D96E000E0220DA6E0650D0
:1019A8000324E16E000E0420E26EDFCFE7FF062A73
:1019B8000550065CD8B01200ECD720EE01F00150BB
:1019C800D9260250DA22DF6A01C0D9FF02C0DAFF45
:1019D800480EDF6E01C0D9FF02C0DAFF000EDB8EB1
:1019E800120064C001F00001625188EC0CF000099B
:1019F800D8B403D001EC0EF01200080E016E040EEC
:101A0800026E89EC0DF0120001C0D9FF02C0DAFFA6
:101A1800DF50036E20EE01F00150D9260250DA2281
:101A2800DF50046E0350016E04C002F01200060E6F
:101A380000018A19D8A403D088C004F001D0046A30
:101A480004C02CF4010E2DEC0DF0010E0001896F7D
:101A58001200016E0001BCB103D0036A080E02D067
:101A6800036A480E026E02C008F401C009F40401BA
:101A7800088F1200000EF2BE010E016EF29E550E86
:101A8800A76EAA0EA76EA68201B002D0F29E01D060
:101A9800F28E12006105D8A404D0BC930401086B2F
:101AA8001200BC83080E016E040E026E89EC0DF064
:101AB8001200606A626A6A6A6B6A6C6A01D065962B
:101AC80065B6FDD7646A666A656A676A8A6B1200DA
:101AD800FF0EEBEC0DF0A50AD8B402D0000E1200F0
:101AE800FF0E026EFF0E7BEC0DF0010E1200036E6E
:101AF80003C0A9FF02C0A8FFA69EA69CA6843EEC30
:101B08000DF0A6B2FED7A694120001C0D9FF02C0FC
:101B1800DAFF040EDF6E01C0D9FF02C0DAFF000E43
:101B2800DB8E12000150D96EDA6A02C0DFFF015065
:101B3800D96EDA6A010ED92603C0DFFF1200076EDC
:101B4800180E016E040E026EC00E036E07C004F07C
:101B580078EC0BF01200140E016E040E026EBF0E2C
:101B6800036E400E046E78EC0BF0120062C08CF02D
:101B7800010E00018B6F01EC0EF0030E0001896F5E
:101B88001200800E9B6E700ED36E100ED26ED2AE07
:101B9800FED7900EB56E1200DA69DB697E6B7F0E98
:101BA800066EC00E056EA1EC0AF0120003C001F02B
:101BB80004C002F00EEC0EF00800F5501200F29E80
:101BC800F29CA3945DEC0DF000EF10F01200016E92
:101BD80001C0A9FFA69EA69CA680A8501200080EC8
:101BE800016E040E026E89EC0DF01200080E016EF3
:101BF800040E026E89EC0DF01200080E016E040E40
:101C0800026EE1EC0CF012000001946B936B906B88
:101C18008F6B1200F86A02C0F7FF01C0F6FF1200CE
:101C280001C072F002C073F01200010E646E65808C
:101C38001200016E01C089F01200BE91BF91C091DF
:101C4800120000018A511200010E806F120040EC50
:101C58000CF0120016EC0BF01200D3EC0BF0120093
:101C6800010E816F1200010EDC6F1200A4EC04F06B
:101C7800120001C087F0120074EC0AF01200000E86
:051C88001200FFFF0146
:061C8E001200120012001A
:101ECE0000C33CAA513CC355AE544B415050303127
:101EDE00A5FA1FEC1F9E1FC01FFA1F6A1F361FC0D8
:101EEE001FF31E080809024300020100C032090454
:101EFE000000010202010005240010010424020268
:101F0E0005240600010524010001070581030A00CE
:101F1E000209040100020A00000007050202400047
:101F2E0000070582024000003403430044004300D2
:101F3E002000520053002D003200330032002000EA
:101F4E0045006D0075006C006100740069006F0043
:101F5E006E002000440065006D006F0034034D00DC
:101F6E006900630072006F00630068006900700012
:101F7E00200054006500630068006E006F006C0066
:101F8E006F0067007900200049006E0063002E008C
:101F9E0022035400450043004B0049004F0020002F
:101FAE005000490043003100380020005500530016
:101FBE0042001A0330003100320033003400350085
:101FCE00360037003800390041004200120100028D
:101FDE0002000008D8040A000001010200010E03ED
:101FEE005400450043004B0049004F000403090410
:011FFE0000E2
:020000040030CA
:0E00000021081F3CFF91A5FF0FC00E800F408E
:00000001FF
